:100000000C94B3030C94EB030C94EB030C94EB03F0
:100010000C94EB030C94EB030C94EB030C94EB03A8
:100020000C94EB030C94EB030C94EB030C9402295B
:100030000C94B1290C94C9230C94EB030C94EB039E
:100040000C94EB030C94EB030C94EB030C945224F0
:100050000C94EB030C94EB030C94EB030C94EB0368
:100060000C94EB030C94EB030C94EB030C94EB0358
:100070000C94EB0391069106BD06BD061E071508FC
:10008000150815083C07A407B507B5077E138113AB
:1000900086138B13901395139A139F13A413AA130B
:1000A000AF13E61D581EEE1DB81DBC1DF21DBF1D71
:1000B000F51D001ECA1D4E1ECE1D041ED21D081E9B
:1000C000321ED61D0C1E3C1EDC1D121E1C1EC31D26
:1000D000F91DC61DFC1DE11D171E281E481E4A1EC7
:1000E000B41DEA1D611E1320192007200D201F20BA
:1000F00025202B20B521B821EF2102220A2215222A
:10010000182218221822602260221D222022252275
:1001100032223F22422246225322192A402A382BD9
:10012000402A382B8C2AAF2A382B062B152B290076
:100130001E001F00200021002200230024002500B3
:10014000260027002D002E0031002B0014001A007D
:100150000800150017001C0018000C001200130006
:100160002F0030002A0039000400160007000900A3
:100170000A000B000D000E000F00330034003100A8
:100180002800E10064001D001B00060019000500A6
:1001900011001000360037003800E5002152E00061
:1001A000E300E20000002C0000002C0000002C0006
:1001B0000000E600E70065002152007C3A003B00A9
:1001C0003C003D003E003F00400041004200430033
:1001D000440045000100010001005200010001003F
:1001E0000100010001000100010001000100010007
:1001F00001000100500051004F000100010001000A
:1002000001000100010001000100010001000100E6
:1002100001000100010001000100010001000100D6
:1002200001000100010001000100010001000100C6
:1002300000000100000001000000010000000100BA
:1002400001000100010001000100010001000100A6
:100250000100010001000100010001000100010096
:100260000100010001000100010001000100010086
:100270000100010001000100010001000100010076
:100280000100010001000100010001000100010066
:100290000100010001000100010001000100010056
:1002A0000100010001000100010001000100010046
:1002B0000100010001000100010001000000010037
:1002C0000000010000000100000001000100010029
:1002D0000100010001000100010001000100010016
:1002E0000100010001000100010001000100010006
:1002F00001000100010001000100010001000100F6
:1003000001000100010001000100010001000100E5
:1003100001000100010001000100010001000100D5
:1003200001000100010001000100010001000100C5
:1003300001000100010001000100010001000100B5
:1003400001000100010001000000010000000100A7
:1003500000000100000001000100010001001E0F6B
:100360000500047F3F1F643214643214783C1E1E63
:10037000140A052223252628292A2C2D2F30323332
:100380003536383A3B3D3E4042434547494A4C4E5C
:100390005051535557595A5C5E6062646668696B88
:1003A0006D6F71737577797B7D7F81838587898A8E
:1003B0008C8E90929496989A9C9E9FA1A3A5A7A894
:1003C000AAACAEAFB1B3B4B6B8B9BBBCBEBFC1C2C4
:1003D000C3C5C6C7C9CACBCCCDCED0D1D2D2D3D457
:1003E000D5D6D7D7D8D9D9DADADBDBDBDCDCDCDC75
:1003F000DCDDDDDDDDDCDCDCDCDCDBDBDBDADAD943
:10040000D9D8D7D7D6D5D4D3D2D2D1D0CECDCCCBC4
:10041000CAC9C7C6C5C3C2C1BFBEBCBBB9B8B6B4E2
:10042000B3B1AFAEACAAA8A7A5A3A19F9E9C9A9872
:10043000969492908E8C8A89878583817F7D7B7943
:10044000777573716F6D6B6968666462605E5C5A24
:100450005957555351504E4C4A4947454342403EE7
:100460003D3B3A3836353332302F2D2C2A29282679
:10047000252322FFAA7F554000010101010101014E
:100480000101020202020202020202030303030349
:100490000303030404040404040405050505050618
:1004A00006060606070707070708080808090909D6
:1004B000090A0A0A0B0B0B0C0C0C0D0D0D0E0E0E7F
:1004C0000F0F0F1010111111121213131414151510
:1004D00016161717181819191A1A1B1B1C1D1D1E82
:1004E0001E1F2020212222232424252626272829D6
:1004F000292A2B2C2D2D2E2F303132323334353604
:100500003738393A3B3C3D3E3F4041424344454603
:100510004748494A4C4D4E4F5051535455565859DF
:100520005A5B5D5E5F616264656668696B6C6D6F86
:100530007072737577787A7B7D7E808283858788F9
:100540008A8C8E8F91939596989A9C9EA0A2A3A533
:10055000A7A9ABADAFB1B3B5B7BABCBEC0C2C4C634
:10056000C9CBCDCFD1D4D6D8DBDDDFE2E4E7E9EBF0
:10057000EEF0F3F5F8FAFDFF0000000000000000C7
:100580002A2B2800000000000000000000000000EE
:1005900000000029000000002C1E342021222434F9
:1005A0002627252E362D3738271E1F2021222324CB
:1005B00025263333362E37381F0405060708090A67
:1005C0000B0C0D0E0F101112131415161718191A03
:1005D0001B1C1D2F3130232D350405060708090A81
:1005E0000B0C0D0E0F101112131415161718191AE3
:1005F0001B1C1D2F3130354C000000000000000096
:1006000000000000000000000000000000000000EA
:100610000000000000000000000000007E0F00D479
:10062000FFFFFFC70000007822035700610066004B
:1006300066006C0069006E00670036003000200024
:100640005200650076002000430000000E033400D5
:10065000700070006C006500740000000403090461
:1006600009025B00030100A0FA0904000001030174
:10067000010009211101000122440007058103083E
:10068000000109040100020300000009211101001A
:100690000122220007058203200001070503032031
:1006A00000010904020001030000000921110100FA
:1006B000012232000705840320000112010002001C
:1006C000000008444408000300010200010660FF26
:1006D0000961A1010962150026FF009520750881B6
:1006E000020963150026FF00952075089102C005D8
:1006F000010980A101850319012AB700150126B758
:1007000000950175108100C0050C0901A101850447
:1007100019012AA002150126A00295017510810079
:10072000C005010906A101050719E029E715002503
:100730000195087501810295017508810105071968
:100740000029FF150026FF009506750881000508A1
:1007500019012905150025019505750191029501DD
:1007600075039101C00011241FBECFEFD4E0DEBF9E
:10077000CDBF04B603FE18C08091DA029091DB026F
:10078000A091DC02B091DD028730904BA740B04BC6
:1007900059F41092DA021092DB021092DC021092ED
:1007A000DD02E0E0F8E3099511E0A0E0B1E0E8EC5B
:1007B000FAE502C005900D92A23FB107D9F722E0F9
:1007C000A2EFB1E001C01D92AA3DB207E1F70E947D
:1007D0004C130C94622D0C9400001F93CF93DF9365
:1007E000D82F0E945205C82F8823A1F0D1FF0CC03A
:1007F0000E946315182F0E946015D82F0E945D1566
:1008000020E0412F6D2F04C020E040E060E080E058
:100810000E9402178C2FDF91CF911F910895282FEE
:100820008430E8F46530D8F44E30C8F4862F90E078
:100830006EE070E00E946F2BFC01822F90E066E476
:1008400070E00E946F2B8E0F9F1FFC01E40FF11DC3
:10085000EE0FFF1FE25DFE4F85919491089581E0B8
:1008600090E0089581E0089581E008950E943404A5
:1008700008950E94360408950E943404089508954E
:100880000E943F040895A6E0B0E0E9E4F4E00C948F
:100890000B2C49835A839E833091F90189819A8177
:1008A000311115C03E81332359F0222349F00E94B3
:1008B000AF09182F682F89819A810E94860903C089
:1008C0000E949B09182F69817A81812F04C00E94A0
:1008D000AF0969817A810E94EC102696E3E00C94BE
:1008E000272CFC01262F40815181628173818481F4
:1008F00095810E9443040895CF93DF93EC0161E05A
:100900000E947104BE010E943904DF91CF910895C5
:10091000CF93DF93EC0160E00E947104BE010E945E
:100920004004DF91CF91089591E001C0990F8A951D
:10093000EAF7892F0E94D0080895CF93C82F81E04D
:100940000C2E01C0880F0A94EAF70E94340E8C2FF7
:100950000E949404CF91089581E008950E94AC0410
:100960000895CF93C82F0E9482088C2F0E94AE0456
:100970002FEF84E39CE0215080409040E1F700C0DD
:100980000000CF91089581E00E94B1040E94782474
:10099000089580E00E94B1040E949C2408950F9362
:1009A0001F93CF93DF938C0161E00E947104EC01EF
:1009B000F801858181110E94681BB801CE010E9457
:1009C000F720882309F45EC0B801CE010E943C04E0
:1009D000882309F457C0B801CE010E94FB1F882369
:1009E00009F450C0B801CE010E94901D882309F47B
:1009F00049C0B801CE010E94661D882309F442C097
:100A0000B801CE010E9468138823E1F1B801CE013C
:100A10000E943E208823B1F1B801CE010E94EA1164
:100A2000882381F1F8018581882341F1C330FCE7F7
:100A3000DF07D1F040F4C115ECE7DE0791F0C130DB
:100A4000DC47A1F01BC0CB358CE7D807A9F0CC352B
:100A5000ECE7DE0771F0CA35DC4781F40E940F0E27
:100A60000DC00E94C3040EC00E94170E0E94C9044C
:100A700009C00E94050E02C00E94130EC8010E9408
:100A8000320401C080E0DF91CF911F910F91089552
:100A90000E94A7230E94580508950E945C050E94A9
:100AA000B023089581E0089508950E94ED0308950C
:100AB00080E00E94550508950E9470220E9455050D
:100AC0000895CF930E947022C82F8091F401C81717
:100AD00079F0C093F4010E9437246093F50170937C
:100AE000F6018093F7019093F8018C2F0E94550531
:100AF000CF910895ADE0B0E0E0E8F5E00C940C2C67
:100B0000488759876A877B878C879D8791110E94C8
:100B1000410DCE01019627E0FC0111922A95E9F7DB
:100B200026E0FE013896DC0101900D922A95E1F74E
:100B30002D8121110AC029813A814B815C816D810F
:100B40007E818F810E94820C04C00E947C048111EE
:100B5000F2CF2D96E2E00C94282CFC012481213068
:100B600021F4808191810E94DC090895CF9388232C
:100B7000D9F1C82F8CEF8C0F813A70F48C2F0E9422
:100B8000E122882329F08C2F0E9424230E94A30DA8
:100B90008C2F0E941C230CC080E28C0F883058F4EC
:100BA000C77081E001C0880FCA95EAF70E94240D42
:100BB0000E94A30D19C0EBE5EC0FE33040F4F0E028
:100BC000E05AFE4F808190E00E9488220DC0C85AF2
:100BD000CB3150F4EC2FF0E0EE0FFF1FE65DFE4F3F
:100BE000808191810E94AD22CF910895882339F1AF
:100BF0009CEF980F913A18F40E9424230DC090E2C4
:100C0000980F983060F4877091E001C0990F8A9531
:100C1000EAF7892F0E942A0D0E94A30D08959BE5F3
:100C2000980F933028F480E090E00E948822089585
:100C3000885A8B3120F480E090E00E94AD22089524
:100C40001F93CF93DF93182FEB010E94B6052097D7
:100C500041F08FE99FE00197F1F700C00000219774
:100C6000F6CF812F0E94F605DF91CF911F91089555
:100C7000893319F060E070E002C060E570E00E9426
:100C800020060895882321F00E94240D0E94A30DC0
:100C90000895882321F00E942A0D0E94A30D089533
:100CA000A0E0B0E0E6E5F6E00C94062C7C01162FFF
:100CB000C72FFC01D581068102950F700E941A0D85
:100CC0008823F9F0DD23E9F08C2F807F803461F0F8
:100CD00080E2810F8830A8F08C2F807E803221F452
:100CE000123078F0002369F08091A90282FF09C0D8
:100CF00082E00E94D90D0E941A0D91E0D82ED926CB
:100D000001C0D12CCC2EC2948FE0C8228C2D90E053
:100D10008C30910508F089C1FC01E65CFF4F0C9412
:100D2000EF2B8C2F807FCF70882311F0C295C07F6E
:100D3000DD2399F0CC2309F464C180E2810F88306F
:100D400010F0111104C08C2F0E94240D03C08C2FB1
:100D50000E94340D0E94A30D54C1812F0E94F605FC
:100D6000CC2309F462C180E2810F883038F111236D
:100D700029F18C2F0E943A0D24C08C2F807FCF70D8
:100D8000803211F0C295C07F112319F0113099F112
:100D90003CC08091A90282FD17C0DD2349F0CC231D
:100DA00029F08C2F0E94240D0E94A30D80E02AC1FF
:100DB00080E00E94F605CC2309F437C18C2F0E94F5
:100DC0002A0D0E94A30D31C1DD2349F0002309F152
:100DD000013009F02AC18C2F0E944B0D26C1011150
:100DE00024C18C2F0E9449068C2F0E94570D8C2FF6
:100DF0000E94AC0D1AC1DD2321F0063008F015C1A8
:100E000008C0053008F011C115C0DD2331F0011113
:100E1000F8C08C2F0E94420608C1002359F01933F4
:100E200009F000C1FFEF27EE83E0F1502040804041
:100E3000E1F7F6C08C2F0E944906F7C08C2F8695EB
:100E40008695837019F0813061F0EFC0DD2321F0C9
:100E5000812F9C2F937002C080E090E00E94882236
:100E6000ECC0DD2321F0812F9C2F937002C080E025
:100E700090E00E94AD22E1C08C2F837079F5D111F2
:100E8000D8C0412F429546954770440F440F212FFB
:100E90002F70042E01C0220F0A94EAF714FF08C035
:100EA0008FE090E001C0880F4A95EAF7809501C075
:100EB00080E0C695C695C370822BC23049F058F4C5
:100EC000C13019F00E94D908B4C00E94D308B1C043
:100ED0000E94DF08AEC00E94D008ABC0DD2319F02D
:100EE0008C2F817001C08695882309F4A2C0412F00
:100EF000429546954770440F440F212F2F70042EC2
:100F000001C0220F0A94EAF714FF08C08FE090E0B6
:100F100001C0880F4A95EAF7809501C080E0C69528
:100F2000C695C370822BC23049F058F4C13019F015
:100F30000E9425097EC00E941F097BC00E942B09C8
:100F400078C00E94E80875C0CF70DD2339F08C2F7F
:100F50000E94FA08812F0E9442066BC0812F0E94D6
:100F600049068C2F0E94060964C0123F21F128F423
:100F7000103F41F0113FC1F040C0133F19F1143F41
:100F800079F03BC0DD2341F0053008F04EC08C2FD6
:100F90008F710E94130949C0063008F046C0F7CF90
:100FA0008091A90282FD18C0DD2339F08C2F8F714A
:100FB0000E94FA083AC0DD23C9F38C2F8F710E947A
:100FC000060933C0DD2329F08C2F8F710E94F108B0
:100FD0002CC00E94ED0829C0DD2331F063E08C2F86
:100FE0008F710E94BB0D21C081E00E94D90D02309B
:100FF000E0F082E00E94D90D18C0DD2331F000231B
:10100000A9F2812F0E94B60510C00023B1F2193356
:1010100049F49FEFE7EEF3E09150E040F040E1F754
:1010200000C00000812F0E94F60588EF8C0D8430EF
:1010300020F40E9470220E945505DD2089F00E9454
:10104000160D80FD0DC0F70115820E94100D0E9443
:10105000FA08C7010E944D080E94100D0E9406095F
:10106000CDB7DEB7E8E00C94222C0F931F93CF93FB
:10107000DF93EC01688179818D810E94E7098C0101
:101080000E9431090E94C308B801CE010E94500697
:10109000DF91CF911F910F910895CF93DF93FC01C2
:1010A00024812223D1F0EC010E94CF0481110FC0D2
:1010B0000E941A0D882389F08D81882371F0809118
:1010C000A90282FF0AC082E00E94D90D06C0CE01AB
:1010D0000E943508CE010E948804DF91CF910895C7
:1010E00080E090E00E94882280E090E00E94AD22A3
:1010F0000E94410D0E94A30D08950E942C230E947E
:10110000700808950E94310D0E947D0808959295FF
:101110009F70963079F010F4925001C09A5092303E
:1011200068F4803F69F018F4883E40F409C0843FB9
:1011300029F406C0883E20F0813F11F080E0089538
:1011400081E00895FC012481222339F0808191817E
:101150000E94DC090E948708089580E00895A6E0B7
:10116000B0E0E5EBF8E00C940C2C2696E2E00C9451
:10117000282CA7E0B0E0EFEBF8E00C940C2C2796BD
:10118000E2E00C94282C089508950E94C408089564
:101190000E94C50808950E94C80880931602089509
:1011A0000E94CB08089590911602892B0E94CB08CB
:1011B00008959091160289230E94CB08089590917A
:1011C000160289270E94CB0808950E94C40808953A
:1011D0000E94E50880931502089580E00E94E808C7
:1011E000089591E001C0990F8A95EAF7892F0E942E
:1011F000E808089521E030E001C0220F8A95EAF75F
:1012000080911502822B0E94E808089521E030E0C9
:1012100001C0220F8A95EAF720958091150282235A
:101220000E94E808089521E030E001C0220F8A956D
:10123000EAF78091150282270E94E80808959091AC
:101240001502892B0E94E8080895909115028923C0
:101250000E94E80808959091150289270E94E808E5
:1012600008950895282FFA01862F8770A1E001C004
:10127000AA0F8A95EAF7CB0133E0969587953A95C0
:10128000E1F763E070E00E946F2BE80FF91F40E088
:1012900050E0622F70E090819B01042E02C03695D1
:1012A00027950A94E2F72170219529272A232927D7
:1012B00021934F5F5F4F4330510569F70895FB015C
:1012C000A82FA77023E0969587952A95E1F763E00C
:1012D00070E00E946F2BE80FF91F40E050E080E0C3
:1012E000219130E00A2E02C0369527950A94E2F744
:1012F00021703327042E01C0220F0A94EAF7822BB3
:101300004F5F5F4F4330510559F70895953090F482
:101310008E3080F4362F282F892F90E06EE070E019
:101320000E946F2BBC01620F711D4AEF51E0832FA9
:101330000E9432090895953080F48E3070F4282F81
:10134000892F90E06EE070E00E946F2B6AEF71E0F1
:10135000820F911D0E945F09089580E00895CF9249
:10136000DF92FF920F931F93CF93DF936C01009155
:10137000150280911602082BC3E0D0E010E0C801EE
:101380000C2E02C0959587950A94E2F780FD04C063
:101390002197A8F7F12C07C0FC2EB6018C2F0E94D4
:1013A000F8100197A9F38F2DDF91CF911F910F9125
:1013B000FF90DF90CF900895CF93DF93EC010E94D0
:1013C000AF09BE010E94F810DF91CF9108951F93DD
:1013D000CF93DF93EB019091F901992321F0CB0199
:1013E0000E94DC0913C0882349F0CB010E94AF0999
:1013F000182F682FCE010E94860904C0CB010E94DD
:101400009B09182FBE01812F0E94F810DF91CF9108
:101410001F910895E1E0F0E0DF0102C0AA0FBB1FB9
:101420006A95E2F7BD01DF0102C0AA0FBB1F4A9512
:10143000E2F7AD01462B01C0EE0F2A95EAF7942F93
:101440009823491302C08E2B0895E0958E230895AA
:10145000242F462F682F809115020E940A0A0E94AD
:10146000E8080895CF93DF93C09117028091180286
:10147000C817A9F0D0E0CE0167E070E00E946F2BA2
:10148000FC01E75EFD4F20813181428153816481FF
:10149000758186810E94B9082196C770E7CFDF91D8
:1014A000CF91089520915102309152024091530200
:1014B00050915402609155027091560280915702EA
:1014C0000E94B9080895CF93DF93809157028295C7
:1014D0008F7009F04CC080915602882309F447C0F0
:1014E0002091170240911802A0915202B09151022E
:1014F000C0915302D09154022417C9F130E0C901C0
:1015000067E070E00E946F2BFC01E75EFD4F848175
:10151000882349F181818A1326C080818B1323C0DF
:101520008581811120C0828193818C1B9D0B883C19
:101530009105C8F4809157028F70806180935702A3
:10154000C90167E070E00E946F2BFC01E15EFD4F76
:1015500090819F709061908381E592E00E944D0898
:101560000E94320A04C02F5F3F4F2770C5CFDF9122
:10157000CF910895CF93B82FC62F20911702A09135
:1015800018022A17B1F030E0C90167E070E00E944C
:101590006F2BFC01E75EFD4F81818C1306C08081BB
:1015A0008B1303C08581841306C02F5F3F4F2770C4
:1015B000E8CF80E001C081E0CF910895A4E1B0E0E0
:1015C000E4EEFAE00C94022C8C0186E0F801DE01D6
:1015D0001F9601900D928A95E1F7F8018481E580CC
:1015E00091E5A92E92E0B92E90915502911118C063
:1015F000882309F480C1EE20D9F1C8010E94A20815
:10160000F82E8823A9F187E0F801D50101900D9209
:101610008A95E1F7C5010E94AD050E94630A98C052
:10162000F801C080D18082809380F0905602209192
:10163000530230915402A401421B530BFF2009F4C2
:1016400006C1483C510508F0AFC0882309F455C1D4
:1016500080915702282F207F90915202222361F01F
:101660009D1509F462C0C8010E94A208811173C0CF
:10167000C8010E944D083FC19D1115C090915102B3
:101680009C1111C0E1100FC08F70806180935702D0
:101690000E94520A81E592E00E944D088091570213
:1016A000F801868326C1E1103AC040E06D2D8C2DF3
:1016B0000E94BA0A40E06D2D8C2D0E94BA0AE82ED5
:1016C000811117C1CF86D88A8F8598890E94DC093D
:1016D000292F22952F70243020F49F70223028F07B
:1016E00009C02A50223080F014C0992349F081119A
:1016F00007C013C0992321F0F8019681907F69F00B
:10170000805E883030F409C0803F38F0815F8330DC
:1017100020F0C8010E944D08EF2CFE2CEEC08091F5
:101720005702816080935702E4C0909151029C114E
:101730009ACFE11098CFF8018683C8010E944D0826
:1017400087E0F801A1E5B2E001900D928A95E1F7FA
:101750000E94520AD2C0EE2009F48ACF209157028B
:10176000822F82958F7090E002978CF080915102C9
:1017700090915202998788879B868A86809155022C
:101780008C871D862E87CE0108960E944D0887E023
:10179000F801A1E5B2E001900D928A95E1F70E946F
:1017A000630A0E94520AA7C090915702292F207FF6
:1017B000A1F4682D9A8A898AA6017A899E2D0E94B1
:1017C000AF0881E592E00E944D0887E0F501119293
:1017D0008A95E9F70E94520A8CC0882309F48DC0CB
:1017E000809152028D1111C0809151028C110DC057
:1017F000E1100BC0F8019683C8010E944D0887E0F4
:10180000F50111928A95E9F778C0C8010E94A208F3
:10181000882309F42DCFEE2009F42ACF2091570216
:10182000822F82958F7090E002970CF4B0CF809158
:101830005102909152029A8389839C828B8280917B
:1018400055028D831E822F83CE0101969ECF483C88
:10185000510508F040C0882309F44DC0FE2CEE204D
:1018600009F406CF809152028D1127C08091510258
:101870008C1123C09091570290FD16C0892F82953C
:101880008F70282F30E02115310571F0F801968313
:101890002F30310509F451CF8F5F982F9295907FAB
:1018A00086818F70892B48CF87E0F801A1E5B2E0EF
:1018B00001900D928A95E1F720C0C8010E94A2080C
:1018C000811165CF80915702816080935702C801D2
:1018D0000E944D0812C0682D9A8A898AA6017A89C9
:1018E0009E2D0E94AF0887E0F50111928A95E9F7D5
:1018F0002FCFF12C02C0FF24F3948F2D6496ECE0DF
:101900000C941E2CAEE0B0E0E8E8FCE00C940C2C4B
:10191000288739874A875B876C877D878E87CE01CA
:1019200008960E94DE0A882369F06C85662309F414
:101930005FC0288539854A855B857D858E850E94B7
:10194000B90856C087E0FE013896DE011196019075
:101950000D928A95E1F76C85662309F449C0809160
:10196000180290E09C012F5F3F4F27703327409172
:10197000170250E02417350709F441C06D8367E072
:1019800070E00E946F2BDC01A75EBD4F97E0FE0167
:10199000319601900D929A95E1F7209318020E94DA
:1019A000320A26C090E067E070E00E946F2B875EED
:1019B0009D4F0E94DE0A882379F18091170290E002
:1019C00067E070E00E946F2BFC01E75EFD4F208115
:1019D0003181428153816481758186810E94B90879
:1019E0008091170290E001968770992780931702E3
:1019F00080911702909118028913D4CF0DC00E94D4
:101A000082081092180210921702E1E5F2E087E0D6
:101A1000DF011D928A95E9F72E96E2E00C94282CBE
:101A200080916002869586958695089580916002E2
:101A30008770089590916002977081E009F480E0CA
:101A4000089580916C02089590916C02892B809387
:101A50006C020895809590916C02892380936C02AA
:101A6000089510926C02089590916B02892B8093D7
:101A70006B020895809590916B02892380936B028D
:101A8000089510926B02089508950E94440D0895E0
:101A90000E94450D089590916202292F28238217F4
:101AA00029F0982B909362020E94480D089590911E
:101AB0006202292F282331F08095892380936202C6
:101AC0000E94480D089580916202882329F01092A7
:101AD000620280E00E94480D08950F931F93CF93F8
:101AE000DF930091040110910501C0916C02809177
:101AF0006B02C82B80916202882331F0C82B0E94B0
:101B0000D22281110E94630DF801C083C0910401AB
:101B1000D091050148E050E068E572E0CE010E94F6
:101B2000D52C892B59F088E0FE01A8E5B2E00190A0
:101B30000D928A95E1F7CE010E947D22DF91CF912F
:101B40001F910F9108950E946D0D08950E94440DFC
:101B500008950E94A60D089590916102292F2823CF
:101B600031F080958923809361020E94A90D089528
:101B70000E94440D08959091A90292FF11C0982FE0
:101B8000990F990F990F692B609360020E94FA08D0
:101B9000809160028695869586950E94B80D08957D
:101BA0000E94FA0808951092600280E00E94B80D29
:101BB0000895909160028095892380936002282F78
:101BC000277069F4981759F09091A90292FF07C005
:101BD0008695869586950E9406090E94D30D0895E4
:101BE0009091A90292FB222720F9281769F080FB27
:101BF00092F99093A9028091A8029091A9020E9463
:101C00003F0E82E00E94D90D08958091A90282FBC7
:101C1000882780F991E089270E94F00D089581E0DE
:101C20000E94F00D089580E00E94F00D08956FEF7E
:101C30007FEF80E090E00E942D2D089580E090E0FD
:101C40000E94F92C853E9E4F19F40E948920089528
:101C500080E0089582E090E00E94EB2C089583E0FC
:101C600090E00E94EB2C0895682F83E090E00E94A2
:101C70000F2D089584E090E00E94F92C0895BC0196
:101C800084E090E00E942D2D0895AB01BC018FE00F
:101C900090E00E94212D0895AB01BC0183E190E00A
:101CA0000E94212D089560E070E0CB010E944C0E4F
:101CB000089560E070E0CB010E94450E0E94530E33
:101CC0000895A8E0B0E0E7E6FEE00C940C2C65EE89
:101CD0007EEF80E090E00E942D2D60E082E090E0B9
:101CE0000E940F2D81E0809316020E94340E60E066
:101CF00074E184E090E00E942D2D60E086E090E0A9
:101D00000E940F2D60E087E090E00E940F2D40E0E0
:101D100050E0BA0188E090E00E94212D60E083E26B
:101D200090E00E940F2D60E08CE090E00E940F2D6B
:101D300060E08DE090E00E940F2D19821A821B82D4
:101D40001C821D821E821F82188648E050E067E1D7
:101D500070E0CE0101960E94FF2C40E050E0BA01F5
:101D60008FE190E00E94212D80E00E94A2200E943D
:101D7000D7200E94590E2896E2E00C94282C0E944D
:101D8000610E0895682F8EE090E00E940F2D089557
:101D9000A6E0B0E0EEECFEE00C940A2C0E942B24AE
:101DA0008C0180916D0290916E020817190781F0E5
:101DB00019821A820E942B24682F49815A81792F17
:101DC00080E090E00E947A0510936E0200936D020D
:101DD0002696E4E00C94262C0E94372460937D0222
:101DE00070937E0280937F029093800260937902C9
:101DF00070937A0280937B0290937C02089581E035
:101E0000089581E008950E94010F089508950E94A9
:101E1000060F08950E94060F08950E940A0F089564
:101E20000E94060F08950E94100F08950E94060F49
:101E3000089588EE91E10E9463130E94160F0E949C
:101E4000130F08950E94070F0E94060F08950E9425
:101E50001E0E811102C00E94BF0E0E942A0E8093A6
:101E600081020E943A0E9093A9028093A8020E94D8
:101E7000C61B0E942F0E0E94D008809115020E945E
:101E8000E50808950E9422240E94E7200E94BB12C8
:101E90000E94270F0E9454050E94731A0E940D0F82
:101EA0000895A6E0B0E0E7E5FFE00C94002C0E9466
:101EB000FF0E811103C00E94C80E62C00E94D112A1
:101EC0002FE6E22E22E0F22E5701D12CF5010191EE
:101ED00011915F018D2D0E94FD1180279127D394D0
:101EE000F5E0DF1619F0892B89F302C0892B19F36D
:101EF0008091810281FD0E9406120E94030F782EBC
:101F000010E066246394812F0E94FD114C01F701BB
:101F1000A080B180A826B926A114B10449F100E03F
:101F2000CC24C394D12CC5018C219D21892BC1F0D7
:101F30007720B1F009831A830E942B249C838B8322
:101F40006D8221E0C4018C219D21892B09F420E0C0
:101F500049815A816B817C818D81922F0E947A0503
:101F60000F5FCC0CDD1C0E30F1F6F7019182808200
:101F70001F5FF2E0EF0EF11C153029F60E94EC0E07
:101F80000E94691B0E9461052696EEE00C941C2CB1
:101F90001F93CF93DF930E94FD10EC01C11580E5E4
:101FA000D807E8F5C11590E4D90708F0ACC0C03EE9
:101FB000D10530F5CD3CD10508F098C0C83AD1051F
:101FC00078F4C53AD10508F087C0C130D10509F4CD
:101FD00080C008F4F9C0C430D10508F0F8C0F4C0DE
:101FE000C33CD10508F0F0C0C85AD0E0CC0FDD1FCB
:101FF000CD59DE4F0990D881C02DCE019464E8C040
:10200000C11580E2D80708F0D2C0C11591E0D90708
:1020100008F06FC0C83ED10508F4D9C0D5C0C0369D
:1020200082E5D80738F5C03492E5D90708F07DC0BD
:10203000C03282E5D80708F070C0C11592E5D90713
:1020400008F488C04C2F4695469550E0F5E0440FC3
:10205000551FFA95E1F7C37021E030E0C90102C0D5
:10206000880F991FCA95E2F7EA01C82BD92BCE0138
:102070009D68AEC0C03A82E5D807C8F48C2F8F7136
:10208000C03892E5D90708F080C08695869590E023
:1020900065E0880F991F6A95E1F7C37021E030E091
:1020A00002C0220F331FCA95E2F73A686BC0C03CEA
:1020B00082E5D80708F470C0C03E92E5D90708F061
:1020C00083C0CF71DD27DC2FCC27CE01806F906AD3
:1020D0007FC081E090E07CC0C55AD0E0C756DE4F9B
:1020E0008881C82FD0E0CE01906472C0CE01906587
:1020F0006FC08D2F0E949911182FCE0199270E9431
:10210000FD101F715FC0CE0199270E94FD10CC27E2
:10211000DF70D06A8C2B9D2B5BC0CF71D0E0DC2FA1
:10212000CC27CE01816F906A53C08C2F8F7186951A
:10213000869590E09C0175E0220F331F7A95E1F7B8
:10214000C37081E090E002C0880F991FCA95E2F742
:102150009C6818C08C2F8F710E94991195E0D695BC
:10216000C7959A95E1F7CF70D0E0DC2FCC27282FC8
:1021700030E084FF05C084E0220F331F8A95E1F729
:10218000D069CE01822B932B23C090E0D82FCC278F
:10219000CE01846F906A1CC08C2F8F710E949911A0
:1021A0008F7190E0D82FCC27CE01906211C08D2F77
:1021B0008F710E949911182FCE0199270E94FD104E
:1021C0001F719062912B04C080E090E001C0CE01AD
:1021D000DF91CF911F910895753038F46E3028F457
:1021E000462F672F0E947E1C089580E090E008959E
:1021F0000E94EC100E94C80F08958238910569F181
:10220000B0F48133910509F475C048F48932910521
:1022100009F467C08A32910509F471C008958533C5
:10222000910509F459C089339105B9F00895833EA9
:10223000910589F138F4803E9105D1F0823E9105F7
:1022400029F10895863E9105C9F1873E9105D9F19E
:10225000843E910509F06CC027C02091A80220FDA2
:1022600057C021FD55C02091A90223FD5BC00895F0
:102270008091A80280FD48C08091A90280FF48C0DB
:102280008091A80284FD46C083EE51C08091A802CF
:1022900082FF3CC0F5CF8091A80282FD37C08091BB
:1022A000A90280FD35C0ECCF8091A90281FF36C024
:1022B0008091A80284FD2EC087EE39C08091A802CB
:1022C00083FF2AC0F5CF8091A80283FD25C08091AD
:1022D000A90281FD23C0ECCF8091A80285FD22C018
:1022E0001FC08091A80285FD1BC08091A90283FFB9
:1022F00019C00AC08091A80286FD16C017C080913F
:10230000A80286FD13C010C089E311C082EE0FC081
:1023100080EE0DC080E00BC086EE09C084EE07C0E1
:1023200085E305C089E203C08AE201C081E390E051
:1023300008959091A80292FF10C041E0282F2471C7
:10234000243009F040E031E0282F2871283009F0CE
:1023500030E0431711F02CE0822793FF10C041E0DA
:10236000282F2471243109F040E031E0282F287112
:10237000283109F030E0431711F02CE0822730912A
:10238000A90230FF10C051E0282F2171213009F03F
:1023900050E041E0282F2871283009F040E0541720
:1023A00011F029E0822731FF10C041E0282F217170
:1023B000213109F040E031E0282F2871283109F05F
:1023C00030E0431711F029E0822794FD877E0895BD
:1023D00080E00895CF939C01205E32452032310584
:1023E00040F4FB01C581C11105C08F710E949D049D
:1023F00001C0C1E08C2FCF910895E82FF0E0EE0FDF
:10240000FF1FEC54FD4F808191810895089580EA6B
:102410008A95F1F7089500C008950E940712089563
:1024200008950E94101208950E94111208950E94AA
:10243000101208950E9417120895F894E82FE2955B
:10244000EF70F0E031A1282F2F7081E090E001C003
:10245000880F2A95EAF7982F9095932391A392A13C
:10246000892B82A3789408950F931F93CF93DF93C2
:10247000CAEAD1E089918F3F11F00E941D1281E0DC
:10248000CF3AD807B9F7CCE9D1E00AEA11E089914F
:102490008F3F11F00E941D120C171D07C1F7DF912D
:1024A000CF911F910F910895A0E0B0E0EAE5F2E12D
:1024B0000C94052C8C01C62FD0E0CE0186559E4F82
:1024C0006C01FC0190819F3F09F450C0B62EF89436
:1024D000E92FE295EF70F0E081A19F7021E030E0FC
:1024E00001C0220F9A95EAF7822B81A382A1209541
:1024F000282322A378940E940B12ECE9F1E04AEA27
:1025000051E021E030E0E12CF12C61916F3F89F046
:10251000A62FA295AF70B0E090968C9190E06F706E
:1025200002C0959587956A95E2F780FD02C0C901C2
:1025300002C080E090E0E82AF92A220F331F4E17EC
:102540005F0719F7F60180818F3F11F00E941D127D
:1025500061E0E114F10409F460E08B2D0E940D129A
:10256000CC0FDD1FC00FD11FF982E882CDB7DEB7D7
:10257000E9E00C94212C0E9434128AE0E4EBF2E0B2
:10258000DF01982F1D929A95E9F7EAEAF2E0DF0160
:102590001D928A95E9F785E00E940C130E941A1299
:1025A0000895AAE0B0E0E7EDF2E10C94092C8E0169
:1025B0000F5F1F4F8AE0F80111928A95E9F7F12C1D
:1025C0006F2DC8010E945412F394F5E0FF12F8CF6A
:1025D0004AE050E0B8018AEA92E00E94D52C21E05E
:1025E000009709F420E0892B41F08AE0F801AAEA7B
:1025F000B2E001900D928A95E1F745E064EB72E05C
:102600008AEA92E00E940D13182F0E941412812F63
:102610002A96E5E00C94252C0895EF92FF920F93F3
:102620001F93CF93DF937C018B01C42F222351F0A2
:1026300081E0809384020E942B24909383028093F4
:10264000820204C080918402811102C080E01CC01B
:1026500080918202909183020E9443240597B0F3F7
:10266000D0E0CC0FDD1FAE01B701C8010E94D52C10
:10267000892B39F0AE01B701C8010E94E22C81E03C
:1026800001C080E010928402CDB7DEB7E6E00C9482
:10269000242C0E94510F08950E94C8230E941926DD
:1026A0000E94190F0E9433260E94420F0E9440266A
:1026B0000E9445260E9449130E945F260E94F3242F
:1026C0000E94220FF5CF9093F3018093F2010895B9
:1026D0000F931F93CF93FB01C581CC2309F444C012
:1026E0008C010E94210D8272F801E052F847EB3014
:1026F000F105D8F5EA5BFF4F0C94EF2B0E94651AA9
:1027000027C0882329F00E94531A22C08823D9F3B6
:102710000E94431A1DC0882329F00E94A01618C0E9
:102720008823D9F30E94911613C0882329F00E94B0
:10273000C2160EC08823D9F30E94B11609C088239F
:1027400029F00E94E41604C08823D9F30E94D3160E
:10275000C0E00BC0882329F00E943C15F9CF8823E4
:10276000D9F30E941C15F4CFC1E08C2FCF911F919B
:102770000F910895EF92FF920F931F93CF93DF93E2
:10278000E82F71110AC0442321F0F0E0E858FB4F14
:10279000E4916E2F7E2F8E2F6CC0C62FD0E0072FB6
:1027A00010E0282F30E0442329F0F901E858FB4FCE
:1027B000249130E0CE0166E070E00E946F2BEE24A1
:1027C000EA94F12CB7010E94A52BDB01CC0FDD1F91
:1027D000CB016BEA7FEF0E946F2B8C0F9D1FC82FE0
:1027E000CC0FC80FC701801B910BB9010E946F2B42
:1027F000E92F492FD0E0CE01B8010E946F2B692F3D
:1028000070E0C701861B970BB9010E946F2BF92F4F
:10281000C7018C1B9D0BB8010E946F2B692F70E0C4
:10282000C701861B970BB9010E946F2BA230B1051F
:1028300091F040F4109761F01197B9F4722F8E2F38
:10284000EF2F16C0A430B10561F040F0169769F47F
:10285000842F792F0CC0722F892F0AC0822F7F2FCF
:1028600007C0822F7E2FE92F03C08F2F742FE22FF6
:102870006E2FCDB7DEB7E6E00C94242C41E00E9429
:10288000BA13089508950E943E1408959091090185
:10289000291B922FE091DC01F091DD01242F462FBE
:1028A000682F892F90E009950895CF93DF93762FB5
:1028B000E901682F842F0E944314962F672F9E01F1
:1028C000482F892F0E944614DF91CF91089580915F
:1028D000BE02282F2695269530E02115310519F4E2
:1028E0008370846005C02B32310524F08370886AC0
:1028F0008093BE020895A0E0B0E0E1E8F4E10C941A
:10290000062C88E090E00E94F32C6B017C0183E2AE
:1029100090E00E94EB2C282F30E040E050E060E097
:1029200070E080E090E000E20E94332CB22FA32FF1
:10293000F42FE52FD62FC72F97018601BC29A12B95
:10294000F22B5E2F532B2B2F3A2F4F2F6D2F7C2FD7
:10295000CDB7DEB7E8E00C94222CA0E0B0E0E3EBCA
:10296000F4E10C94022C49015A016B017C010E9494
:1029700067148401A4016A2D7B2D88E090E00E94F9
:10298000212D94014A2D5B2DB601C70100E20E9462
:102990004E2C622F83E290E00E940F2DCDB7DEB760
:1029A000ECE00C941E2CEEEBF2E0208131814281B0
:1029B000538164817581868197810E94AD14089549
:1029C000EEEBF2E025E0208311828FEF8283838398
:1029D0001482758130E04FEF5FEF60E08681978170
:1029E0000E94AD1408958091BE0280FF03C08695B9
:1029F0008695089580E008958091BE0281700895C3
:102A00009091C202933018F49F5F9093C202882382
:102A100091F02091BE023091BF024091C0025091CE
:102A2000C1026091C2027091C3028091C402909170
:102A3000C5020E94AD14089581E00E94001508951A
:102A40009091C202992319F091509093C202882369
:102A500091F02091BE023091BF024091C00250918E
:102A6000C1026091C2027091C3028091C402909130
:102A7000C5020E94AD14089581E00E9420150895BA
:102A80008091C20208958093C202662389F0682F64
:102A90002091BE023091BF024091C0025091C1020C
:102AA0007091C3028091C4029091C5020E94AD143E
:102AB000089560E00E94431508958091BF02089533
:102AC0008091C00208958091C10208950F931F93D1
:102AD000CF938091BE0280FF09C0E091E001F091A8
:102AE000E1010995CF911F910F910895C0910B01BC
:102AF0000091DC011091DD0180910C01C81768F78D
:102B0000809109019C2F981B20E040E060E0892F14
:102B100090E0F8010995CF5FEFCFEF92FF920F930E
:102B20001F93CF93DF939091BE0290FF1CC0042FA0
:102B3000162FD82FC0910B01E090DC01F090DD0141
:102B400080910C01C81768F4809109019C2F981B93
:102B5000202F412F6D2F892F90E0F7010995CF5F2E
:102B6000EFCF0E946615CDB7DEB7E6E00C94242CBB
:102B70009091BE0290FF0BC0762F682F842F0E9489
:102B80003E14962F672F482F892F0E948D15089588
:102B9000CF93DF93EC01EC81F0E0ED58FC4F4491D2
:102BA000EEEBF2E0628181810E94B8158C818F5F2B
:102BB0008C83DF91CF910895CF93DF93EC01EEEBFF
:102BC000F2E0438162818C810E94B8158C818F5F15
:102BD0008C83DF91CF910895CF93DF93EC014091E7
:102BE000C1029C8190FF02C0842F01C080E091FF50
:102BF00002C0642F01C060E092FF40E00E948D158A
:102C00008C8190E00196877099278C83DF91CF911A
:102C10000895A0E0B0E0EFE0F6E10C94062C182F48
:102C2000F62E042FE22E9091BE0290FF6AC0E92F8B
:102C3000E695E695AE2FB0E0A155BE4F8C918093FE
:102C400093029C7F943061F4612F7F2D842F0E942A
:102C50003E14962F672F482F892F0E948D153AC05A
:102C6000823019F40091C10235C0863019F41091F8
:102C7000BF0230C08930D9F3893161F5E9518E2F17
:102C80008170D82EE695F0E0ED58FB4FE491C12C11
:102C9000CE2FD0E040910D01C416D0F42C2D30E0A1
:102CA000C901BE010E946F2B642F70E00E94A52B0A
:102CB000812FD11002C0860F01C0861B90910B019D
:102CC000290F311D402F6F2D0E945514C394E2CF60
:102CD0000E9466151093BF02F092C0020093C102D9
:102CE000EE2079F02091BE026091C2027091C30281
:102CF000312F4F2D502F8091C4029091C5020E9418
:102D0000AD14CDB7DEB7E8E00C94222CEEEBF2E088
:102D10009181282F4381628188E0890F0E940916E2
:102D2000089581E00E9486160895EEEBF2E091810D
:102D3000282F4381628188EF890F0E940916089528
:102D400081E00E9495160895EEEBF2E0628128E0A2
:102D5000620F08F46FEF282F438181810E940916CA
:102D6000089581E00E94A4160895EEEBF2E06281DE
:102D700028E0621B08F460E0282F438181810E94D3
:102D80000916089581E00E94B5160895EEEBF2E071
:102D9000438128E0420F08F44FEF282F62818181A0
:102DA0000E940916089581E00E94C6160895EEEB70
:102DB000F2E0438128E0421B08F440E0282F6281C2
:102DC00081810E940916089581E00E94D716089516
:102DD00020E00E94091608959091BE0290FF11C054
:102DE00021110FC0242F462F682F90910901892FA0
:102DF0008195E091DC01F091DD0190E009950E9460
:102E000066150895CF939091BE0290FF0DC0C22F1A
:102E1000762F682F842F0E943E14962F672F2C2F19
:102E2000482F892F0E94EC16CF910895EF92FF92C0
:102E30001F93CF93DF93EC0110E0EE24EA94F12C82
:102E400060910D011617B8F480910B01212F30E02D
:102E5000280F311D70E0C7010E94B92B812F0E94FD
:102E6000662B9C814091C1026091C002890F0E9433
:102E700055141F5FE5CF0E9466159A818C8190FFE3
:102E800002C08F5F01C081508C83DF91CF911F9171
:102E9000FF90EF900895A0E0B0E0E1E5F7E10C9439
:102EA000052CFC01828180FF02C0DFEF01C0D1E070
:102EB000C0E00091DC011091DD0180910D01C81787
:102EC00008F041C080910B0190910901891B8C0F82
:102ED00020E040E060E090E0F801099554E0E52E44
:102EE000F12CB12CCC2ED12C809186028B0D82300E
:102EF00034F487FF05C090910D01890F01C080E077
:102F0000082E000C990BC816D906B1F480910B015C
:102F10009601280F311D8091C10290E0B7010E94F7
:102F20006F2B9595879595958795482F6091C00251
:102F30008091BF020E945514BD0EF1E0EF1AF10816
:102F400099F6CF5FBACF0E94661580918602D13084
:102F500031F4811102C080910D01815007C090E0D1
:102F6000019660910D0170E00E94B92B809386025A
:102F7000CDB7DEB7E9E00C94212C0F931F93CF93CC
:102F8000DF93C0910B010091DC011091DD01809174
:102F90000C01C81768F4809109019C2F981B20E050
:102FA00040E060E0892F90E0F8010995CF5FEFCF16
:102FB00010E0C091DC01D091DD0160910D01161788
:102FC00078F5E12FF0E070E0CF010E94B92B20915D
:102FD0000B01820F20918502022E000C330BE217A9
:102FE000F3079CF020910801022E000C330B2E17E2
:102FF0003F075CF0282F30E04091C1026091C00291
:103000008091BF020E94551409C090910901891B4B
:1030100020E040E060E090E0FE0109951F5FCDCF29
:103020000E9466152091070180918502820F80938E
:10303000850290910801920F9093080119165CF493
:10304000082E000C990B40910D0150E041505109A0
:10305000841795071CF0219520930701DF91CF91EC
:103060001F910F910895A0E0B0E0E9E3F8E10C941E
:10307000FE2B8C01FC01C481CC2ED12CE12CF12C37
:10308000A7019601C701B6010E94802BA7019601F6
:103090000E94802B4B015C0180E290E06C01CC1A15
:1030A000D1080D2C000CEE08FF0825E530E040E0CB
:1030B00050E0C501B4010E94802B2B013C01A70107
:1030C0009601C701B6010E94802BA70196010E94BC
:1030D000802B9B01AC01280D391D4A1D5B1DC301CE
:1030E000B2010E94CD2BD22F822F90E02A3230F0F5
:1030F00025E530E0A901481B590BCA0163E070E0E7
:103100000E946F2B97FD019695958795C82FC095C6
:10311000F12C85E5E82EED1A80910D01F81690F45A
:10312000F1FC02C08E2D01C08D2F90910B012F2D2F
:1031300030E0290F311D4C2F6091C0020E945514C0
:10314000F394EACF0E946615F8018481811102C0D0
:1031500091E003C0803219F49FEF909306019091A3
:103160000601890FF8018483CDB7DEB7E0E10C9446
:103170001A2C0F931F93CF93DF938C01C0E0D0E004
:1031800080910D01282F30E0C217D30734F58695C2
:1031900090E0F801348120910B01C817D9073CF465
:1031A000332371F0CE01820F911D9C0106C03111B5
:1031B00007C0FE01E20FF11D9F014091C10205C051
:1031C000CE01820F911D9C0140E06091C002809170
:1031D000BF020E9455142196D3CF0E946615F801B4
:1031E000848190E00196817099278483DF91CF914B
:1031F0001F910F910895A0E0B0E0E1E0F9E10C9497
:10320000002CFC017280648081E08483E3E7F3E0BA
:103210008490E2EFF3E0E491C091C102C695C158F9
:10322000D0E0CC0FDD1FCD2EDD24912CAA24AA9452
:10323000B12CE8190E2F10E080910D01981608F0BE
:1032400096C0E92CF12C82E0871570F0C70165E08B
:1032500070E00E946F2BFC01E957FD4F8091BF0287
:1032600080838091C0028183C70165E070E00E9485
:103270006F2B611006C0FC01E957FD4F13821282CB
:1032800062C0EC01C957DD4F8B81882321F1815049
:103290008B8390E06FEF70E00E946F2B6C8170E089
:1032A0000E94A52BFB01FF27ED58FC4FE4918E2FC8
:1032B000881990E06FEF70E00E946F2BB8010E94B8
:1032C000A52B2091C10230E0862F90E0B9010E9429
:1032D0006F2B9A8338C00E94B82CB5010E94B92B7D
:1032E0008C159D0584F5E2E0E71588F40E94B82C62
:1032F000B5010E94B92B88830E94B82C2091C0028E
:103300002695622F70E00E94B92B280F2983C701F0
:1033100065E070E00E946F2B89579D4FFC0112827F
:103320002091C102243120F0293C18F028EC01C082
:1033300024E1C70165E070E00E946F2BFC01E957B2
:10334000FD4F2483238380910B019701280F311DAA
:10335000C70165E070E00E946F2BFC01E957FD4F4B
:103360004281618180810E945514939465CF0E94AF
:103370006615CDB7DEB7EEE00C941C2CEEEBF2E058
:1033800020812E7F20833181428153816481758128
:10339000868197810E94AD14109294020E94661556
:1033A0000895EEEBF2E080818E7F8083109294028C
:1033B0000E94661508956091BE026695669570E05C
:1033C0004BE050E08EE091E00E94C82C892B19F46C
:1033D00081E0809394020E942B2490938D0280932D
:1033E0008C0208959091BE0290FF3FC093708111AE
:1033F00002C0946007C08B3210F0986A03C0880F37
:10340000880F982B9093BE02662391F02091BE0204
:103410003091BF024091C0025091C1026091C2023E
:103420007091C3028091C4029091C5020E94AD14B4
:103430006091BE026695669570E04BE050E08EE0CC
:1034400091E00E94C82C892B19F01092940202C0BE
:103450000E94DB1981E080938F024091C10260914C
:10346000C0028091BF020E94E8160895682F9091D3
:10347000BE029695969581E0890F8B3208F081E027
:103480000E94F219089581E00E94361A0895682F6B
:103490009091BE02969596958FEF890F09F48AE276
:1034A0000E94F219089581E00E94471A089561E090
:1034B0000E94F2190895EEEBF2E080818160808332
:1034C000869586950E94571A08958091BE0280FFC6
:1034D00003C00E94BE1908950E945B1A089560E01F
:1034E0000E94F21908958091920281113CC00E94BD
:1034F0007B142093BE023093BF024093C0025093CE
:10350000C1026093C2027093C3028093C40290937D
:10351000C5022C7FA1F40E94E0140E947B1420932A
:10352000BE023093BF024093C0025093C102609329
:10353000C2027093C3028093C4029093C5020E949A
:10354000671410929402E091DA01F091DB01099581
:103550008091BE0280FF04C0869586950E946F1AF6
:1035600081E0809392020895EEEBF2E08081816029
:103570008083869586950E946F1A08958091BE0279
:1035800080FF03C00E94D11908950E94B41A0895C3
:103590000F931F93CF93DF9380919402882309F4B4
:1035A00092C080919302E091BE02E695E695E81BF9
:1035B000E0938E02823049F4F0E0E159FC4FE4914F
:1035C000CE2FD0E008EC15E159C0863049F4F0E088
:1035D000E459FC4FE491CE2FD0E00CED15E14EC044
:1035E000893051F4E695F0E0E759FC4FE491CE2F95
:1035F000D0E006E117E142C08F3051F4E695F0E0EB
:10360000EA59FC4FE491CE2FD0E00BE417E136C02D
:10361000853149F4F0E0ED59FC4FE491CE2FD0E034
:103620000DEB17E12BC08831D9F0833239F4E1E694
:10363000F3E0C591D4910CEE15E120C08432A9F0DD
:103640008532C1F48E2F63E00E94992BE92FF0E0C0
:10365000E25AFC4FE491CE2FD0E00BEF18E10EC000
:10366000C8E2D0E003E318E109C0C4EFD1E009EB00
:1036700018E104C0C0EDD7E002E414E180918F02AC
:10368000882361F010928F020E942B2490938D0268
:1036900080938C0210929102109290020E942B242F
:1036A000E0918C02F0918D028E1B9F0B8F3F9F4704
:1036B00050F4EC0FFD1FF0938D02E0938C028CE828
:1036C00092E0F8010995DF91CF911F910F91089534
:1036D00008950E94C81A0895539A0895362F63E0FA
:1036E00070E00E946F2BDC01AA53BD4F11963C93F2
:1036F00011974C93FD0122830895E6ECF2E081835B
:103700006083428308958BB1877F9BB198602FB708
:10371000F894E6ECF2E032E0E93CF30789F031910D
:1037200048E09BB9000000C037FF8BB9330F0000A1
:1037300000C000C000C08BB900C04A9591F7EBCF24
:103740002FBF8FE594E00197F1F700C000000895C6
:103750000E94170E089580E00E94FD118170089567
:103760000E94D1122FEF86E791E0215080409040D7
:10377000E1F700C000000E94D1120E94AB1B882319
:1037800021F00E94A81B0E94782408950E94B01B7B
:10379000089584E00895E82F862F90E06CE170E0B2
:1037A0000E946F2B242F30E0220F331F280F391F68
:1037B0008E2F90E06CE870E00E946F2B820F931FB9
:1037C000889608950F931F93CF93DF938430A0F4CE
:1037D000653090F44E3080F40E94CB1B8C010E9427
:1037E000EB2C90E0D82FCC27C80101960E94EB2C3F
:1037F0009E01282BC90102C080E090E0DF91CF91AB
:103800001F910F9108950F931F93CF93DF938430EF
:1038100080F4653070F44E3060F4E9010E94CB1BF7
:103820008C016D2F0E940F2D6C2FC80101960E94F4
:103830000F2DDF91CF911F910F9108951F93CF937B
:10384000DF93D0E0C0E010E0412F6C2F8D2F0E945D
:103850000F049C01412F6C2F8D2F0E94031C1F5FB2
:103860001E3091F7CF5FC53071F7DF5FD43051F76D
:10387000DF91CF911F910895EF92FF920F931F93C5
:10388000CF93DF93EA017A01E60EF71E8C01C8019F
:103890008896CE15DF0569F0003322E0120720F488
:1038A0000E94EB2C888301C0188221960F5F1F4F66
:1038B000EECFCDB7DEB7E6E00C94242CEF92FF926A
:1038C0000F931F93CF93DF93EA017A01E60EF71E61
:1038D0008C01C8018896CE15DF0559F0003322E02F
:1038E000120718F468810E940F2D21960F5F1F4F59
:1038F000F0CFCDB7DEB7E6E00C94242C843038F45A
:10390000653028F44E3018F40E94E21B089580E0E0
:1039100090E0089580E1089588EA91E00895EF929B
:10392000FF920F931F93CF93DF93EA017A01E60E84
:10393000F71E8C01C801885A9D4FCE15DF0569F02E
:10394000083A21E0120720F40E94EB2C888301C082
:10395000188221960F5F1F4FEDCFCDB7DEB7E6E09F
:103960000C94242CEF92FF920F931F93CF93DF932D
:10397000EA017A01E60EF71E8C01C801885A9D4FB4
:10398000CE15DF0559F0083A21E0120718F46881D6
:103990000E940F2D21960F5F1F4FEFCFCDB7DEB7DF
:1039A000E6E00C94242CCF93DF93C8E5D2E060E0EE
:1039B000CE010E940F2D2196C11584E0D807B9F7DA
:1039C000DF91CF910895A8E0B0E0E9EEFCE10C941E
:1039D000022CF82E8FE08F1508F474C08FEF93E05F
:1039E0000E94EB2C81116EC008E512E0FF2071F0FF
:1039F000011594E0190709F465C0C8010E94EB2C79
:103A0000811101C0FA940F5F1F4FF0CFFE01319674
:103A10006F0188E011928A95E9F77801FFEFEF1ABC
:103A2000FF0AC8010E94EB2C89831A82882309F4BB
:103A300049C0813009F040C0580182E0A80EB11C95
:103A4000C7010E94EB2C8A838823E1F19FEF980F36
:103A5000933060F4780193E0E90EF11CC5010E94F7
:103A6000EB2C8B83882371F11C8226C0843019F5DE
:103A70004E01E3E08E0E911C02E010E07501FFEFB5
:103A8000EF1AFF0AC5010E94EB2CF40181934F014C
:103A90008823C1F08C3741F4E2E0F0E0EC0FFD1F29
:103AA000E00FF11F108208C00F5F1F4F5701073052
:103AB000110521F707C0750160E0C6010E942C1FA7
:103AC0008701ABCF2896ECE00C941E2CCF93DF93AC
:103AD00086319C4709F5EB010E94210D9D819923B8
:103AE00071F08A7A91E009F490E090939502811147
:103AF00002C089E201C085E30E941C2309C08091B5
:103B00009502811102C089E201C085E30E9424234D
:103B10000E94A30D80E001C081E0DF91CF91089564
:103B2000CF93DF93FC01DB0115968C91882309F478
:103B3000DDC09F0130572332310508F0D8C0EF01B6
:103B40000E943A0E9093A9028093A802FE01E150D0
:103B5000F047E232F10520F4EF5AFF4F0C94EF2BBF
:103B60008091A8028160AAC08091A9028860B2C039
:103B70008091A8028260A2C08091A80220C080919A
:103B8000A80288609BC08091A9021EC08091A902F2
:103B90008260A0C08091A802806190C08091A8023C
:103BA00080628CC08091A802806488C00E948208D4
:103BB0008091A802806882C08091A8028860846099
:103BC0007DC08091A9028260816084C08091A8023A
:103BD0008E7F74C08091A902877F7CC08091A802EB
:103BE0008D7F6CC08091A80220C08091A802877F41
:103BF00065C08091A9021EC08091A9028D7F6AC014
:103C00008091A8028F7E5AC08091A8028F7D56C0F5
:103C10008091A8028F7B52C00E9482088091A802E6
:103C20008F774CC08091A802877F8B7F47C080919F
:103C3000A9028D7F8E7F4EC08091A80282FB222731
:103C400020F991E0922790FB82F990FB83F936C02E
:103C50008091A902982F909591708E7F892B90FB6F
:103C600081F938C08091A80286FB222720F991E0D3
:103C7000922790FB86F922C00E9482088091A802B8
:103C800087FB222720F991E0922790FB87F916C045
:103C900081E001C080E00E94C20E1EC08091A80297
:103CA00084FB222720F991E0922790FB84F906C03B
:103CB0008091A802982F909590FB80F98093A8029C
:103CC0000BC08091A90283FB222720F991E0922763
:103CD00090FB83F98093A9028091A8029091A90298
:103CE0000E943F0E0E94820880E001C081E0DF91C7
:103CF000CF9108958F929F92BF92CF92DF92EF92D1
:103D0000FF920F931F93CF93DF93E82FF0E0E858D3
:103D1000FA4FB490282F26952695269530E0F90184
:103D2000E85EF94FE4908770F12C082E02C0F594FC
:103D3000E7940A94E2F791E0E922FF24F901E85FB1
:103D4000F94FC490D12C082E02C0D594C7940A9480
:103D5000E2F7E1E0CE22DD24F901E850FA4FC49108
:103D6000D0E002C0D595C7958A95E2F7C170DD27EE
:103D7000062F10E0E114F10471F081EE0E94B60507
:103D8000C801009741F0EFE9FFE03197F1F700C07B
:103D900000000197F6CFC114D10439F44801B801ED
:103DA0008B2D0E942006C8010EC086EE0E94B6052B
:103DB000C801009799F3EFE9FFE03197F1F700C0F0
:103DC00000000197F6CF009741F0EFE9FFE031974F
:103DD000F1F700C000000197F6CFCD2819F5EF28C4
:103DE00079F081EE0E94F6050115110549F08FE981
:103DF0009FE00197F1F700C0000001501109F4CFD6
:103E0000CD2BF1F08CE20E94380681149104C1F0B0
:103E1000EFE9FFE03197F1F700C00000F1E08F1A01
:103E20009108F3CF86EE0E94F605C8010097B9F21B
:103E3000EFE9FFE03197F1F700C000000197F6CFFE
:103E4000DF91CF911F910F91FF90EF90DF90CF9076
:103E5000BF909F908F900895EF92FF921F93CF9302
:103E6000DF93EC01162F8881882309F455C0813037
:103E700009F04DC08981813041F47E0182E0E80E75
